:100000000C9462000C94551A0C94821A0C948A0079
:100010000C948A000C948A000C948A000C948A0038
:100020000C948A000C948A000C948A000C948A0028
:100030000C948A000C94BC060C948A000C948A00E0
:100040000C94AF1A0C948A000C94021E0C943D1E62
:100050000C948A000C948A000C948A000C948A00F8
:100060000C9440050C948A00000000002400270036
:100070002A0000000000250028002B0000000000DE
:1000800023002600290004040404040404040202DA
:100090000202020203030303030301020408102007
:1000A0004080010204081020010204081020000012
:1000B0000007000201000003040600000000000029
:1000C0000000E51F11241FBECFEFD8E0DEBFCDBF7B
:1000D00012E0A0E0B1E0E0EDF1E402C005900D9285
:1000E000A43DB107D9F714E0A4EDB2E001C01D9220
:1000F000AD3BB107E1F710E0C4ECD0E004C02297BB
:10010000FE010E94E220C23CD107C9F70E942A20CA
:100110000C94E6200C940000FB01DC0102C001906D
:100120000D9241505040D8F708958091D40281300B
:1001300019F482E08093D4028091D402833019F4C0
:1001400084E08093D4020895E3E0F0E089E08093B6
:100150005700849190E08670863009F491E0892FF1
:1001600008951F93182F0E94A400882379F09FB749
:1001700081E080930304F894A89588E1809360005F
:1001800010936000112309F0A8959FBF1F91089557
:10019000382F20E080910404909105048227932752
:1001A00040E061E270E19C01220F331F97FF04C021
:1001B000C9018627972701C0C9014F5F483099F7C9
:1001C000909305048093040408958436910520F4E7
:1001D000BC0180E090E025C08E3B910550F48A552B
:1001E0009040BC0180E090E02AE030E040E050E048
:1001F00016C0823D910550F4845B9040BC0180E0C4
:1002000090E024E630E040E050E009C08D5C904092
:10021000BC0180E090E028E532E040E050E00E9440
:10022000392024E630E040E050E00E943920089573
:1002300090E08C599F4F0E94E5000895DC0198964C
:10024000EC91F0E0E770F070E454FD4F8081089588
:10025000FC0120A530E0C9018170907001962770E3
:10026000307035952795820F931F880F880F08955A
:100270008F929F92AF92BF92CF92DF92EF92FF92B6
:100280000F931F938C010E941E01D80197962C9109
:1002900030E043E150E0249FF001259FF00D349FB2
:1002A000F00D1124E051FE4F80809180A280B38038
:1002B00090E00F96AA2797FDA095BA2FBC01CD011B
:1002C00020E43FE14DE750E00E943920A501940170
:1002D0000E946C2069017A0180ED97E0A0E0B0E017
:1002E000C80ED91EEA1EFB1ED80198968C91887103
:1002F00081F060E07EEE8AEB9BE0A50194010E9414
:100300006C2028513C4F4F4F5F4FC20ED31EE41E4E
:10031000F51E87EE93E0A0E0B0E0C80ED91EEA1EFD
:10032000FB1EC701B60128EE33E040E050E00E941A
:100330006C20CA01B90128EE33E040E050E00E9491
:1003400039201F910F91FF90EF90DF90CF90BF90D9
:10035000AF909F908F9008951F93182FDB01FA01A3
:10036000482F469530E0848190E083709070982FFC
:1003700088272081820F911D11969C938E938481F2
:1003800090E08C70907076E0880F991F7A95E1F775
:100390002181820F911D13969C938E9312978481D5
:1003A00090E08073907064E0880F991F6A95E1F780
:1003B0002281820F911D15969C938E9314978481B0
:1003C00090E0807C9070880F991F880F991F23817F
:1003D000820F911D17969C938E93169735961896BB
:1003E0003F5F431708F0BFCF10FF50C08081829558
:1003F00086958695837090E02DE431E0AC01429FB4
:10040000C001439F900D529F900D11240C961196A0
:100410009C938E93808190E044E0969587954A95D1
:10042000E1F783709070AC01429FC001439F900D33
:10043000529F900D11240C9613969C938E931297B5
:10044000808190E0969587959695879583709070BA
:10045000AC01429FC001439F900D529F900D11240B
:100460000C9615969C938E931497808190E08370E0
:100470009070AC01429FC001439F900D529F900D20
:1004800011240C9617969C938E9316971F9108959E
:1004900023E08032920718F420E030E026C023E009
:1004A000883E920748F49C012F51334054E0369522
:1004B00027955A95E1F719C027E0803D920720F46F
:1004C0009C012C5D334011C028E08839920718F058
:1004D0002FEF33E00AC09C01285C374044E036959A
:1004E00027954A95E1F72D503C4FC90108958C306E
:1004F000910548F49C0174E0220F331F7A95E1F7CF
:10050000285D3C4F17C023E0843F920720F49C01F4
:1005100024523C4F0FC024E08030920718F020E9AD
:1005200038E008C09C012657334F64E0220F331F88
:100530006A95E1F7C90108959C01369527952575BF
:100540003575821B930B9C0136952795369527951B
:100550002373337383739373280F391FC901E4E046
:1005600096958795EA95E1F7820F931F8F709F709C
:1005700021E031E0AC01429FC001439F900D529FAA
:10058000900D1124892F0895882339F04298000096
:10059000419A0000429A0000089542980000419854
:1005A0000000429A00000895429A000086B14298E5
:1005B0000000817008950F931F93082F5C9A429852
:1005C0005C9810E0802F80780E94C402000F1F5FAB
:1005D0001830C1F742981F910F9108958F770E94AC
:1005E000DB0208950F931F93082F10E0802F80786F
:1005F0000E94C402000F1F5F1830C1F742981F917C
:100600000F9108950F931F93429880E000E0182FF8
:10061000110F0E94D402810F0F5F0830C1F71F91A4
:100620000F9108950E94EE020E9402035C9A0895C1
:100630001F93162F80680E94DB02812F0E94F20216
:100640005C9A1F9108951F931091F9021827E0EF0B
:10065000F2E0E80FF11D89E767850E9418038DE33A
:10066000612F0E94180382E4612F0E9418031F91DA
:10067000089586E20E94120308950F931F938BE260
:100680000E941203082F8CE20E941203282F30E0F0
:1006900016E0369527951A95E1F710E0000F111F27
:1006A000000F111F202B312BC9011F910F910895AD
:1006B0000F931F938C018CE1F80164810E94180351
:1006C0008DE1F80165810E9418038EE1F8016681D1
:1006D0000E94180380E2F80167810E94180381E2FA
:1006E000F80160850E94180382E2F80161850E948A
:1006F000180383E2F80162850E94180384E2F8017E
:1007000063850E94180385E2F80164850E9418033E
:100710008AE2F80165850E9418038EE6F801668575
:100720000E9418038FE6F80167850E94180380E78E
:10073000F80160890E94180381E7F80161890E942D
:10074000180382E7F80162890E9418031F910F9134
:100750000895EF92FF920F931F93CF93DF937B0146
:100760008C01603028E372072CE982072CE19207A4
:1007700028F520E836E948E950E00E946C20E901BC
:100780006897B90180E090E020E839E647E65FEF3E
:100790000E9439206E0D7F1D801F911F22E0660F81
:1007A000771F881F991F2A95D1F721E732E040E093
:1007B00050E00E946C20890180E421C020E03DE2ED
:1007C00041E351E00E946C20E9016897B90180E0A3
:1007D00090E020E033ED4EEC5EEF0E9439206E0D8C
:1007E0007F1D801F911F660F771F881F991F21E7AC
:1007F00032E040E050E00E946C20890180E69E01DA
:100800002F71622F680F85E70E94180386E7612F1A
:100810000E94180387E7602F0E941803CDB7DEB748
:10082000E6E00C94D1209F92AF92BF92CF92DF92DC
:100830000F93DF93CF9300D000D0CDB7DEB7982EC3
:1008400083E00E9412038093190384E00E94120344
:1008500080931A0386E060E00E94180387E061E05D
:100860000E94180389E06FE70E9418038AE065E0A0
:100870000E9418038BE062E10E9418038CE065E19E
:100880000E9418038DE06DEF0E9418038EE060E077
:100890000E941803992019F08FE492E008C080911B
:1008A000170323E1829FC001112480519E4F0E94B3
:1008B000580380E36CE80E94180382E36FE00E9413
:1008C000180383E362E40E94180384E36AE00E9451
:1008D000180385E36AE20E94180386E36DE20E9432
:1008E000180387E364ED0E94180388E360E00E9428
:1008F000180389E360E00E941803992049F055E845
:10090000A52E51ECB52E51ECC52E5EEDD52E08C0AE
:10091000A090F902B090FA02C090FB02D090FC02C5
:100920000AE38D2D9927AA27BB2789839A83AB8356
:10093000BC83802F69810E941803802F8B5F69819F
:100940000E941803DC2CCB2CBA2CAA240F5F0E3388
:1009500041F783E46FEF0E94180384E46FEF0E9475
:10096000180385E46FEF0E94180386E46FEF0E947E
:100970001803992019F08DE666E003C08DE66091BA
:10098000FD020E94180389E760E00E9418038AE7CD
:100990006091FE020E94180383E760E00E94180342
:1009A00084E760E00E941803992029F060EC7AEC5B
:1009B00089E896E308C06091F5027091F602809193
:1009C000F7029091F8020E94A9030F900F900F90E8
:1009D0000F90CF91DF910F91DF90CF90BF90AF90AC
:1009E0009F90089587E061E00E9418038EE764E21B
:1009F0000E94180388E063E00E94180388E060E02A
:100A00000E94180387E065E00E94180385E062E019
:100A10000E94180383E00E9412038093190384E06C
:100A20000E94120380931A03089590E0411191E00F
:100A3000880F982B9093BA00660F6093BD00309397
:100A4000200320931F030895882311F085EC01C033
:100A500085E88093BC00089585ED8093BC0080916B
:100A6000BC0084FDFCCF089585EC8093BC00089504
:100A7000ECEBF0E0108285E480831092250308956A
:100A80001F920F920FB60F9211242F933F934F9303
:100A90005F936F937F938F939F93AF93BF93EF93E6
:100AA000FF93DF93CF930F92CDB7DEB78091B9005C
:100AB00090E0887F90708036910509F4EAC0813615
:100AC0009105CCF58832910509F47CC089329105F5
:100AD000B4F48031910509F470C0813191053CF482
:100AE000009709F40EC1089709F00DC166C088315E
:100AF000910509F467C0809709F005C177C080347B
:100B0000910509F490C08134910544F48033910536
:100B100009F46EC0C89709F0F6C06CC08035910525
:100B200009F471C08835910509F483C088349105B2
:100B300009F0E9C0A5C08839910509F4DCC08939FC
:100B40009105ECF48837910509F4A3C08937910524
:100B50004CF48836910509F49CC08037910509F062
:100B6000D2C097C08838910509F4C5C08039910575
:100B700009F492C08038910509F0C5C08DC0803B52
:100B8000910509F4A5C0813B91054CF4803A91058B
:100B900009F499C0883A910509F0B5C099C0803C24
:100BA000910509F4AAC0883C910509F4A6C0883BC8
:100BB000910509F0A8C080E08CC08091210380934A
:100BC000BB009BC0809124038150809324038F5FDE
:100BD00009F43FC0E0912203F091230381918093B7
:100BE000BB00F0932303E093220387C082E049C057
:100BF00083E047C084E080932603809125038B7FA8
:100C00008093250362C08091BB00E0912203F091A4
:100C100023038193F0932303E09322038091240321
:100C200081508093240380912403823008F065C0B2
:100C300062C08091BB00E0912203F0912303819375
:100C4000F0932303E0932203809124038150809347
:100C50002403809125038B7F8093250380912503B6
:100C600080FF4FC0809125038E7F80932503809164
:100C7000250382608093250384EA8093BC0043C0EF
:100C800085E080932603809125038B7F8093250345
:100C900038C01092240331C0E0911F03F09120036B
:100CA000309749F19091BB00809124038F5F80932E
:100CB0002403815011F060E001C062E09983CE010D
:100CC000019609951BC00E942C050E9434051BC08B
:100CD00081E0E0911F03F0912003309761F08823B9
:100CE00011F461E001C063E0CE010196099599819C
:100CF0009093BB0003C080E001C081E00E94240506
:100D000002C00E942C050F90CF91DF91FF91EF91CF
:100D1000BF91AF919F918F917F916F915F914F9113
:100D20003F912F910F900FBE0F901F90189525B1F6
:100D300090E0FC01EE0FFF1FE80FF91FE557FC4F95
:100D40008081282B25B988B19181892B88B98BB1F5
:100D50009281892B8BB9089585B19091BB0389232A
:100D600085B988B19091BC03892388B98BB19091E2
:100D7000BD0389238BB908951F920F920FB60F926E
:100D800011241F932F933F934F935F936F937F9300
:100D90008F939F93AF93BF93CF93DF93EF93FF9383
:100DA00010915E0380918602C0918402D0918502E9
:100DB000181708F05BC08091BE039091BF03909319
:100DC000870080938600E12FF0E0EE0FFF1FEE59C1
:100DD000FD4F808191810E947702880F991F909327
:100DE000BF038093BE038091BE039091BF039E0119
:100DF000281B390BC901309385022093840220916E
:100E0000EB023091EC02220F331F8217930720F47C
:100E1000309385022093840280916003882339F403
:100E20008091E30280FF59C0183008F456C08FEF5C
:100E30009FEF909389008093880080918400909127
:100E400085008097D0F30E94AC0680915F038823D1
:100E500039F480915E03882319F081500E9497062F
:100E600080915E038F5F80935E033EC08091BE03DE
:100E70009091BF039093870080938600D093BF0327
:100E8000C093BE0380916003882319F08FEF9FEF1A
:100E900006C08091BE039091BF0388559240909305
:100EA00089008093880080E49CE990938502809378
:100EB000840280918400909185008097D0F30E94F5
:100EC000AC0680915F03882329F4809186028150CB
:100ED0000E94970610925E0307C08091BE03909116
:100EE000BF0388559240A5CFFF91EF91DF91CF913D
:100EF000BF91AF919F918F917F916F915F914F9132
:100F00003F912F911F910F900FBE0F901F9018953A
:100F100090E0880F991F880F991F8C30910518F465
:100F20002CE030E007C09C0183E0253F380710F03B
:100F300024EF33E0C9010895809162039091630327
:100F40008F5F9F4FE9F08091E402482F50E0A2E6C6
:100F5000B3E020E030E02417350761F0F8948D917C
:100F60009C911197F901EE0FFF1FEE59FD4F9183F0
:100F7000808378942F5F3F4F12962031310559F7C7
:100F800008951F93CF93DF93EC0170E0CB01827043
:100F9000907060FF1AC0892B31F0809184038883A0
:100FA0001092020445C01091020480EF92E00E946A
:100FB0001E011817D8F5E12FF0E0E054FC4F8081B6
:100FC00088831F5F1093020433C0892BC1F098817E
:100FD0009093010410920204892F807E803651F490
:100FE00080918403823010F188818F718093430354
:100FF00083E01AC09E3FE1F41092840317C08091F1
:1010000001048F3FA9F420910204293278F4E22FE1
:10101000F0E0E051FD4F88818083822F8F5F8093C5
:101020000204893229F481E08093840380E001C0C6
:1010300081E0DF91CF911F910895EF92FF920F937E
:101040001F93CF93DF9380E260E040E021EC37E034
:101050000E94150510928403E2E0EE2E75E0F72E53
:1010600004E080918403813039F480E00E9413040D
:10107000E09284034398F5CF10918403133061F418
:101080002D98809143030E9423031093D4020E9461
:10109000F20400938403E5CF80918403843009F740
:1010A0008091D4028430E9F68FE70E94EE02C0E01E
:1010B000D0E007C00E940203FE01E054FC4F808391
:1010C000219680EF92E00E941E0190E0C817D90798
:1010D0008CF3F09284032D9AC4CFA0E0B0E0E3E754
:1010E000F8E00C94B120EC010E94051B5B016C013F
:1010F0007E0100E010E011C0209779F00E94051BEE
:101100006A197B098C099D09E616F7060807190775
:1011100020F40E94380581E008C08091250382FDFB
:10112000EBCF8091260310922603CDB7DEB7EAE01D
:101130000C94CD20A0E0B0E0E0EAF8E00C94B320FD
:10114000182F7B01042FC22FD0E0F4E0CF2ED12C3A
:10115000CC22DD2222FF03C080E090E004C0809119
:101160008202909183020E946D08282F8823B9F58E
:101170001092260300932403F0922303E0922203AB
:10118000110F11601093210390912503C1FD02C03E
:1011900084E001C085E0892B80932503809125039D
:1011A00081FF0BC0809125038D7F80932503809163
:1011B00021038093BB0085EC01C085EE8093BC00C9
:1011C000C0FF0DC0C114D10419F080E090E004C04C
:1011D00080918202909183020E946D08282F822FB5
:1011E000CDB7DEB7E8E00C94CF20A0E0B0E0EBEFA5
:1011F000F8E00C94B320182F7B01042FC22FD0E00D
:10120000A4E0CA2ED12CCC22DD2222FF03C080E034
:1012100090E004C080918202909183020E946D0848
:10122000282F8823B1F51092260300932403F0920F
:101230002303E0922203110F1093210390912503C1
:10124000C1FD02C084E001C085E0892B80932503A5
:101250008091250381FF0BC0809125038D7F8093B2
:101260002503809121038093BB0085EC01C085EEAE
:101270008093BC00C0FF0DC0C114D10419F080E000
:1012800090E004C080918202909183020E946D08D8
:10129000282F822FCDB7DEB7E8E00C94CF208091C5
:1012A000D402813011F081E008950E94051B209145
:1012B0001B0330911C0340911D0350911E03621BC0
:1012C000730B840B950B615A76488140904010F463
:1012D00080E0089582E00895FF920F931F93CF93CB
:1012E000DF93182F092FF62E8EE30E941803212F6B
:1012F000302FC901EC0110E005C08FE769910E9411
:1013000018031F5F1F15C8F385E064E00E941803EF
:1013100083E00E9412038093190384E00E94120369
:1013200080931A030E94051B60931B0370931C0398
:1013300080931D0390931E0387E069E00E941803C9
:1013400081E08093D402CDB7DEB7E5E00C94D220E3
:101350000E946C098091D4028130D9F40E94051B4F
:1013600020911B0330911C0340911D0350911E03DB
:10137000621B730B840B950B605A7648814090403A
:1013800040F4E8CF8BE994E060E071E00E94ED1D4D
:1013900008958091D4028130A9F30895A1E0B0E0CE
:1013A000E4EDF9E00C94B920809184038230B9F423
:1013B00080E2BE016F5F7F4F41E021E00E949A080A
:1013C000882379F08FEF809384030E94F71A60934B
:1013D00085037093860380938703909388038FEF30
:1013E00001C089812196E2E00C94D520A1E0B0E013
:1013F000ECEFF9E00C94B920809184038230D9F4A9
:1014000080914303805A898380E2BE016F5F7F4FE2
:1014100041E021E00E94F508882369F08FEF809376
:1014200084030E94F71A6093850370938603809368
:101430008703909388032196E2E00C94D520AAE2DA
:10144000B0E0E5E2FAE00C94B7208FEF8983DE018B
:101450001296E0EFF2E089E201900D928150E1F7FF
:1014600080E28E010F5F1F4FB8014AE221E00E9427
:10147000F508882351F480E2B80141E021E00E94A0
:101480009A08882311F482E001C08FEF80938403CF
:1014900080918403823051F00E94F71A6093850393
:1014A000709386038093870390938803AA96E4E061
:1014B0000C94D320A2E0B0E0E0E6FAE00C94B52072
:1014C0000E94051B9B01AC0180912703909128038A
:1014D000A0912903B0912A0379018A01E81AF90A37
:1014E0000A0B1B0BD801C70181519742A040B040A5
:1014F00008F444C080912B038F5F80932B038150AD
:1015000080FD02C000E001C007E020932703309374
:1015100028034093290350932A038BE994E063E066
:101520000E94A51F8BE994E061E00E94A51F47E09F
:10153000F42EF00E802F90E0880F991F9C012E59F9
:101540003D4F3A832983F90160817181672F7727A5
:1015500063707070880F991F682B792B8BE994E06A
:101560000E94A51FE981FA816081718170708BE909
:1015700094E00E94A51F0F5F0F15E1F62296E6E0AA
:101580000C94D1201F93182F8BE994E0612F0E94B7
:10159000A51F812F0E94C8001F910895A0E0B0E010
:1015A000E4EDFAE00C94B320082F0E94051B9B0188
:1015B000AC018091270390912803A0912903B09159
:1015C0002A0369017A01C81AD90AEA0AFB0AD70173
:1015D000C60181519742A040B04008F443C0209317
:1015E0002703309328034093290350932A03109232
:1015F00005041092040488EA0E94C20A002311F430
:1016000081E001C081E80E94C20A80E10E94C20A12
:10161000C0E0D0E0FE01EE0FFF1FEE59FD4F8081CC
:1016200091810E9477028C0153E0000F111F5A959F
:10163000E1F7812F0E94C20A802F0E94C20A2196E0
:10164000C031D10539F7609105048BE994E00E941F
:10165000A51F609104047091050470708BE994E0FB
:101660000E94A51FCDB7DEB7E8E00C94CF20A0E024
:10167000B0E0EDE3FBE00C94B320182F062F0E949E
:10168000051B9B01AC018091270390912803A09139
:101690002903B0912A0369017A01C81AD90AEA0A12
:1016A000FB0AD701C60181519742A040B04008F41F
:1016B000D6C12093270330932803409329035093E6
:1016C0002A038091620290916302880F991F809390
:1016D0002C03977080912D03887F892B80932D0395
:1016E0002091640230916502220F331F922F990FCF
:1016F000990F990F8770892B80932D03422F429564
:101700004695477080912E03807C932F9770990F98
:10171000990F990F842B892B80932E0320916602B9
:1017200030916702220F331F922F9295990F990FD4
:10173000907C8F73892B80932E03932F9295990F12
:10174000990F907C822F86958695892B80932F0305
:10175000932F969596959170809130038E7F892B6B
:10176000809330032091680230916902220F331F69
:10177000922F990F8170892B80933003422F441F41
:101780004427441F80913103807F932F9770990FD6
:10179000842B892B8093310320916A0230916B0254
:1017A000220F331F922F9295907F8F70892B8093F9
:1017B0003103422F42954F70809132038078932FEE
:1017C00097709295907F842B892B80933203209180
:1017D0006C0230916D02220F331F8F77809332039A
:1017E000932F979599279795822F8695892B80938C
:1017F0003303932F96959370809134038C7F892BBC
:101800008093340340916E0250916F02440F551F34
:10181000942F990F990F8370892B80933403942F01
:10182000929596959695937020913503207E852FFD
:101830008770880F880F292B282B209335038091E0
:10184000700290917102880F991F382F3295330FD3
:10185000307E2F71232B20933503292F2295220FC1
:10186000207E869586958695822B8093360380917F
:10187000720290917302880F991F809337039770BB
:1018800080913803887F892B8093380320917402DC
:1018900030917502220F331F922F990F990F990FD4
:1018A0008770892B80933803422F42954695477065
:1018B00080913903807C932F9770990F990F990F1E
:1018C000842B892B80933903209176023091770203
:1018D000220F331F922F9295990F990F907C8F733F
:1018E000892B80933903932F9295990F990F907CB0
:1018F000822F86958695892B80933A03932F969510
:101900009695917080913B038E7F892B80933B034A
:101910002091780230917902220F331F922F990F74
:101920008170892B80933B03422F441F4427441F1F
:1019300080913C03807F932F9770990F842B892B84
:1019400080933C0320917A0230917B02220F331F57
:10195000922F9295907F8F70892B80933C03422F1A
:1019600042954F7080913D038078932F97709295A8
:10197000907F842B892B80933D0320917C023091B2
:101980007D02220F331F8F7780933D03932F97950E
:1019900099279795822F8695892B80933E03932FC5
:1019A0009695937080913F038C7F892B80933F03A2
:1019B00040917E0250917F02440F551F942F990F42
:1019C000990F8370892B80933F03942F929596955E
:1019D0009695937020914003207E852F8770880F05
:1019E000880F292B282B209340038091800290910F
:1019F0008102880F991F382F3295330F307E2F7157
:101A0000232B20934003292F2295220F207E869599
:101A100086958695822B80934103112311F490E0E3
:101A200001C098E0002311F480E001C084E0892B1C
:101A3000809342038BE994E06FE00E94A51FCCE203
:101A4000D3E08BE994E069910E94A51F83E0C33441
:101A5000D807B9F78BE994E060E00E94A51FCDB7E5
:101A6000DEB7E8E00C94CF201F93182F8091DE02A0
:101A70008B3221F48CE0612F0E94001C8091D602F1
:101A8000873259F4112321F08091B000806103C0A6
:101A90008091B0008F7E8093B0001F9108950F93C6
:101AA0001F9380915C0390915D039F770E949C023D
:101AB000982F8F3029F4809158038695805804C060
:101AC00089E0989FC0011124809359030091E4029A
:101AD000003170F4F89410E0809159030E94880757
:101AE000000F111F0E591D4FF801918380837894C8
:101AF0008091D6028132C9F490915903892F815087
:101B00008E3F60F08091B0008F7D8093B00060E0E8
:101B1000911161E083E00E94001C07C09093B40023
:101B20008091B00080628093B0001F910F91089562
:101B30001F93182F811111E082E1612F0E94001C78
:101B400083E1612F0E94001C109224031092250350
:101B50008091B9008C6F8093B90080E28093B800C7
:101B600085E48093BC001F910895CF93DF938BE9A8
:101B700094E00E94321F892BF9F08091FF03C82F57
:101B8000D0E09E012F5F3F4F2F7130708091FE0398
:101B900090E02817390781F08BE994E00E946C1FD0
:101BA000C252DC4F88838091FF0390E001968F71D1
:101BB00090708093FF03DBCFDF91CF910895EF9278
:101BC000FF921F93CF93DF9380EF92E00E94280152
:101BD000809386029091E402981719F49F5F909386
:101BE0008602EBE8F3E0108211821282339623E042
:101BF000E23BF207C1F78FEF8093BB038093BC03F6
:101C00008093BD03E6EDEE2EE2E0FE2EA5E9B2E004
:101C1000E7016FEF5FEF4FEF88818031F0F490E0E4
:101C20003C91FC01EE0FFF1FE80FF91FE557FC4F39
:101C30008081832B808311962C9111978181822B37
:101C4000818312969C9112978281892B8283309591
:101C5000432320955223909569232196139682E081
:101C6000C33ED807C9F66093BD035093BC034093AD
:101C7000BB03C8E8D2E010E0F7018081823238F07F
:101C80008632B0F0863219F4888160E00FC01B30D4
:101C900021F48091C1008F7E05C01C3029F4809111
:101CA000C100877F8093C100888161E00E94941BFE
:101CB0001F5F0894E11CF11C21961D30E9F680910C
:101CC000DB02803231F489E061E00E94001C82E88E
:101CD00001C082E08093800081E080935F03809365
:101CE00060038091D602813211F08732C9F483E01B
:101CF00061E00E94941B83E060E00E94001C8091E0
:101D0000D602813221F481E08093B00009C082E0E4
:101D10008093B00085E08093B1008EE38093B300A0
:101D20008AE1809381008FEF9FEF909389008093E9
:101D3000880080ED97E0909387008093860080E490
:101D40009CE990938502809384029093BF038093D3
:101D5000BE0310925E0380916F00816080936F00DC
:101D60008091E30283FF0DC0809162039091630331
:101D70008F5F9F4F31F00E949C071092600310927A
:101D80005F03DF91CF911F91FF90EF9008958EE058
:101D900060E00E94941B8FE061E00E94941B80E150
:101DA00061E00E94941B82E060E00E94941B84E04A
:101DB00061E00E94941B089583E00E9412038093C7
:101DC000190384E00E94120380931A0387E061E004
:101DD0000E9418036AE070E080E090E00E942B1BF4
:101DE0000E94F204000008950F931F93082F17C05C
:101DF000439A64E670E080E090E00E942B1B4398D9
:101E000064E670E080E090E00E942B1B1F5F1017DB
:101E100078F36CE271E080E090E00E942B1B10E010
:101E2000F6CF482F392F25E00DC0F999FECF1FBA04
:101E3000842F932F92BD81BD60BD0FB6F894FA9A9E
:101E4000F99A0FBE215059F0F999FECF842F932FA4
:101E500092BD81BDF89A80B5681739F7089582E080
:101E60000E94F40E0895A0E0B0E0E9E3FFE00C94D6
:101E7000AB20482E562EEE24FF24C0E0D0E0CC2428
:101E8000DD248824992404C055245394CC24DD24D3
:101E9000442051F485EDE82E82E0F82EC0E0D0E039
:101EA0000BE1802E912C19C021E0421651F410EF65
:101EB000E12E12E0F12ECDE1D0E0B9E28B2E912C93
:101EC0000CC032E0431649F4A2E6EA2EA3E0FA2E53
:101ED000C8E4D0E0F0E28F2E912C3E016C0C7D1C0A
:101EE0001092050410920404E3011BC0552059F41C
:101EF000F999FECFD2BDC1BDF89A80B5F701E00FC8
:101F0000F11F808307C0F701E00FF11FCE01608150
:101F10000E94110F0E0D1F1DF80180810E94C80044
:101F200021969E012619022F10E008151905F0F2DE
:101F3000CE015520D9F4F999FECFD2BDC1BDF89A92
:101F400020B5F999FECF2196D2BDC1BD2197F89A4F
:101F500080B590E0B22EAA248A299B2920910404FE
:101F6000309105042817390759F48ECF21966091D6
:101F700005040E94110FCE01609104040E94110F0C
:101F800080E091E0C80ED91E91E0C91693E0D90611
:101F900008F47ECF852DCDB7DEB7E0E10C94C720E5
:101FA00082E060E00E94330F882331F48FEF9FEFCF
:101FB0009093630380936203089582E061E00E943E
:101FC000330F0895282F81E08093D50281E280931A
:101FD000D602E7EDF2E080E081938F5F8830E1F791
:101FE00086E28093DF028093E00284E28093E10244
:101FF00085E28093E20282E08093E3028FEF809398
:10200000E4029AE09093ED021092EE021092EF0239
:102010001092E5021092E6021092E7021092E80296
:102020008EE18093E9029093EA0288EB9BE0909323
:10203000EC028093EB02222361F080E061E00E94D9
:10204000330F8FEF9FEF90936303809362030E949F
:10205000DD0F0895ADE5B0E0E0E3F0E10C94A920D8
:102060005B016C010E94F71A1B012C0181E00E94A8
:10207000130483E08093D4020E94DC0E8BE994E089
:102080006CE071E00E94ED1D3E010894611C711C22
:10209000E3C08BE994E06AE171E00E94ED1D8FE7F7
:1020A0000E94EE020E940203182F8983823601F5F6
:1020B00000EF12E00E940203F80181938F01F3E028
:1020C00009311F07B9F78091F002873309F0BFC0CB
:1020D0008BE994E063E271E00E94ED1D82E4898364
:1020E000CE01019661E00E94A8092D9A81E0CAC044
:1020F000803719F0893631F506C020E52A83AA24F5
:10210000BB24650105C081E00E94E20F89E48A8357
:1021100080910304882321F08091E302806803C04A
:102120008091E3028F778093E302DE011396E5ED61
:10213000F2E08BE101900D928150E1F7CE01029621
:102140006CE183C08437D9F434E53E8F83E08F8F10
:1021500090E798A3EDE0E9A3EAA3DE019396E6ED0C
:10216000F1E08AE101900D928150E1F7CE014E96A7
:102170006FE10E94A809AA24BB24650168C08537C5
:1021800091F405ED12E00E940203F80181938F01A2
:10219000F2E0003F1F07B9F780E061E00E94330FD3
:1021A00025E5298350C0863631F5809162039091F0
:1021B00063038F5F9F4FD1F086E48DAF92E6E92EE7
:1021C00093E0F92E8E01025C1F4FF70181919191EE
:1021D0007F010E947702F801908381830E5F1F4F79
:1021E000F2E8EF16F3E0FF0681F701C01DAFCE0164
:1021F000CD9661E22AC08736D9F402E613E00E9448
:102200000203982E88240E9402039401280F311D96
:10221000C9010E944802F801819391938F01F3E074
:1022200002381F0761F727E429830E94DD0F0BC0E6
:10223000873469F48FEF9FEF909363038093620379
:102240000E94DD0F1983C30161E00E94A80993E099
:102250009093D4020E94F204A114B104C104D104E9
:1022600059F00E94F71A62197309840995096A15D1
:102270007B058C059D0528F48091D402843061F79C
:1022800008CF80E0C35ADF4FE2E10C94C52080E024
:1022900060E00E94330F882319F481E00E94E20F6E
:1022A000089581E061E00E94330F089581E060E0CD
:1022B0000E94330F882311F490E006C090E08091D3
:1022C000F002873309F491E0892F0895EF92FF928D
:1022D0000F931F93CF93DF93EB019C01442737FDAE
:1022E0004095542F60E271EA87E090E00E948E20D2
:1022F00089011216130614F001E010E0BE018827D0
:1023000077FD8095982F20E231EA47E050E00E9467
:1023100039209801442737FD4095542F0E948E2084
:102320007901C0E0D0E009C0419AC8010E944F1B6A
:102330004198C8010E944F1B2196CE15DF05A4F3DA
:10234000CDB7DEB7E6E00C94D1202D9A83E00E9451
:1023500012038093190384E00E94120380931A03EE
:1023600086E060E00E94180387E061E00E941803A5
:1023700089E06FE70E9418038AE065E00E94180375
:102380008BE062E10E9418038CE065E10E94180373
:102390008DE06DEF0E9418038EE060E00E9418034C
:1023A00080E76CE20E94180380E360E00E9418035B
:1023B00089E760E00E9418038AE765E00E9418033D
:1023C00081E762E10E94180382E762E00E9418033D
:1023D00083E760E00E94180384E760E00E9418032E
:1023E0006091E5027091E6028091E7029091E80227
:1023F0000E94A9038DE667E00E9418036AE070E07E
:1024000080E090E00E942B1B87E069E00E941803A7
:102410006AE070E080E090E00E942B1B88E891E089
:1024200061E070E00E946611A8958DE665E00E946B
:1024300018036AE070E080E090E00E942B1B88EBBC
:1024400091E061E070E00E946611A8958DE664E07D
:102450000E9418036AE070E080E090E00E942B1B6D
:102460008DE591E061E070E00E946611A8958DE62F
:1024700062E00E9418036AE070E080E090E00E9451
:102480002B1B8FEA90E061E070E00E946611A89536
:102490008DE660E00E9418036AE070E080E090E062
:1024A0000E942B1B85E091E062E070E00E946611C3
:1024B000A89587E061E00E9418032D980895A6E191
:1024C000B0E0E5E6F2E10C94AB20A8958CE00E9428
:1024D0001203882359F48BE994E06EE271E00E94C4
:1024E000ED1D80E00E9413040E94DC0E0E94B50DD9
:1024F0000E94051B0E94CE09B82E8E010F5F1F4F50
:10250000AA24AA948091D402843029F045E0E42ED4
:10251000BE1409F096C10E94051B6B017C018091DD
:10252000D4028430E9F48FE70E94EE0200E010E06C
:1025300008C00E940203F801E054FC4F80830F5F43
:102540001F4F80EF92E00E941E0190E008171907CC
:1025500084F30E943D0390935B0380935A0328C049
:1025600080EF92E00E941E01482F4F5F80E2B80189
:1025700021E00E949A08882369F0A09284030E94B7
:10258000F71A609385037093860380938703909373
:102590008803B8CF80EF92E00E941E01482F20EC04
:1025A00033E0FE013296C901BF0150E00E948C0069
:1025B000C0924403D0924503E0924603F092470351
:1025C0001092830380915C0390915D03880F991FA3
:1025D000816090935D0380935C0343982D9A80E023
:1025E0000E94340D8091C003282F30E0C9018E7302
:1025F0009070892B09F041C0F8948091180387707E
:1026000062E672E041EC53E00E94AC010091E4020A
:10261000003160F410E0809159030E948807000F98
:10262000111F0E591D4FF80191838083789480917A
:10263000C00390918A0380FF1BC0992309F045C015
:10264000A2E6B3E020E030E0F901EE0FFF1FEE5903
:10265000FD4F808191818D939D932F5F3F4F20315E
:10266000310591F70E94DD0F81E080938A032DC030
:10267000992359F110928A0328C0C9018873907078
:10268000C89719F54091D503842F822787FF1DC075
:1026900040584093D5038091E2028532B1F410E0B6
:1026A0000AC01F5FE12FF0E0E054FC4F8BE994E09B
:1026B00060810E94A51F212F30E08091C00390E02F
:1026C000877090708217930764F780918203882344
:1026D00019F481E0809382031092610310925F03EA
:1026E0001092600380911803887109F4A1C0409191
:1026F000D5038091C00390E0242F30E082279327F8
:1027000086FD60C0407C80E448274093D5039091CB
:10271000FE038091FF03981701F1A6EDB3E030E0CE
:102720000FC03F5F892F90E0FC01E252FC4F2081F7
:102730002D9301968F7190708093FE03383031F0A5
:102740009091FE038091FF03981759F7395C8091AF
:10275000D503382B3093D50335C080915703809330
:10276000D6038091DF02863251F482E10E94631C1D
:1027700095958795959587958093D70302C010927C
:10278000D7038091E002863251F483E10E94631CFA
:1027900095958795959587958093D80302C010925B
:1027A000D80380915B038093D90380915A0380936F
:1027B000DA0380915C0390915D039F770E949C02F5
:1027C0008093DB0385ED93E069E00E946C0902C011
:1027D0000E94B50D0E944F098823D1F306ED12E047
:1027E00058E8E52E52E0F52EF8018081E82FF0E060
:1027F000CF01807F9070409791F4EF70F070EE0FF2
:10280000FF1FEE59FD4F8081918160E08F3F910560
:1028100011F008F061E0F70180810E94001C0F5F59
:102820001F4F0894E11CF11CF2E0033E1F07E1F684
:1028300083E08093D4020E94F20481E080938903B4
:102840002D980E94051B5B016C010E94F71A2B0159
:102850003C0180918303823008F065C0E09044031E
:10286000F09045030091460310914703809148037F
:1028700090914903A0914A03B0914B038E159F0597
:10288000A007B10709F44FC080EF92E00E94380121
:10289000A60195012E193F09400B510B6C5D754047
:1028A000804090406217730784079507E0F5E09237
:1028B0004803F092490300934A0310934B030E948C
:1028C0003903809357032091550330915603280F05
:1028D000311D3093560320935503609154036F5F6D
:1028E000609354036930F8F0C90170E00E945820E9
:1028F000CB0170935603609355032091580343E036
:10290000249F90011124820F931F96958795969589
:102910008795809358030E944F0D10925603109292
:1029200055031092540380918203909000048823F1
:1029300009F457C180908303891408F0D5C180EF52
:1029400092E00E9438012091440330914503409168
:10295000460350914703A21AB30AC40AD50A685124
:102960007C4F8F4F9F4F6A157B058C059D0508F0A6
:1029700075C080915C0390915D03880F991F9093BF
:102980005D0380935C0381E080938903882081F458
:1029900040924C0350924D0360924E0370924F034D
:1029A000109250031092510310925203109253034D
:1029B000809183038F5F8093830380EF92E00E9476
:1029C00038012091440330914503409146035091D2
:1029D0004703260F371F481F591F20934403309386
:1029E0004503409346035093470381E08093890356
:1029F000439A0E94340D0E944F0D30C080EF92E048
:102A00000E9438019B01AC018091440390914503E1
:102A1000A0914603B091470386017501E81AF90AAF
:102A20000A0B1B0B682D70E080E090E00E943920BB
:102A30006E157F058007910788F410925D03109250
:102A40005C0381E0809389030E944F0DA0924403B0
:102A5000B0924503C0924603D0924703809183030E
:102A6000882309F4E8C09091ED02992389F18091BF
:102A70006103882369F5892F90E00E94E500209189
:102A80004C0330914D0340914E0350914F0383010D
:102A90007201E21AF30A040B150B6E157F0580070D
:102AA0009107B0F481E0809361030E949C078091BC
:102AB000E9020E941801640D751D861D971D616055
:102AC0006093500370935103809352039093530388
:102AD0009091EF029923F1F080915F038823D1F464
:102AE000892F90E00E94E50020914C0330914D0326
:102AF00040914E0350914F0383017201E21AF30A91
:102B0000040B150B6E157F058007910718F481E003
:102B100080935F039091EE029923F1F0809160031E
:102B20008823D1F4892F90E00E94E50020914C0386
:102B300030914D0340914E0350914F038301720138
:102B4000E21AF30A040B150B6E157F058007910737
:102B500018F481E0809360038091E5029091E60291
:102B6000A091E702B091E8020097A105B10509F430
:102B700062C08091500390915103A0915203B09193
:102B800053030097A105B10509F455C083017201F3
:102B9000E81AF90A0A0B1B0B17FD4DC06091EA02F7
:102BA00070E080E090E028EE33E040E050E00E94EA
:102BB00039206E157F0580079107E8F50E94A51161
:102BC00080E00E9413040E94F2040E94F71A6160E0
:102BD0006093500370935103809352039093530377
:102BE0002AC080EF92E00E9438019B01AC018091E5
:102BF000440390914503A0914603B0914703860199
:102C00007501E81AF90A0A0B1B0B692D70E080E0C8
:102C100090E00E9439206E157F058007910758F4D7
:102C2000A0924403B0924503C0924603D09247035A
:102C300081E080938903809160038823B1F48091BF
:102C4000E202883219F40E945A0A0FC0893239F41C
:102C500080916103609183030E94370B06C08A3222
:102C600021F4809161030E94CE0A80918903882318
:102C7000B9F0E0914303EF5FE0934303E83131F0B3
:102C8000F0E0E051FD4F8785882311F41092430353
:102C9000809143030E9423030E94F6091092890346
:102CA000809184038F3F21F50E94F71A20918503BC
:102CB000309186034091870350918803621B730B08
:102CC000840B950B695E73408040904088F00E94B1
:102CD000F71A60938503709386038093870390931C
:102CE00088030E941F0A04C0891409F0B7CE86CE5B
:102CF0006696E0E10C94C720FF920F931F93082F74
:102D0000F62E61E00E94941B802F61E00E94001C5F
:102D10008F2D61E00E94001C8AE090E00E944F1B12
:102D20008F2D0E94331C892B11F410E00FC0802FCF
:102D300060E00E94001C8AE090E00E944F1B8F2DF3
:102D40000E94331C10E0892B09F411E0802F60E011
:102D50000E94941B802F60E00E94001C8F2D60E079
:102D60000E94001C812F1F910F91FF900895EF92F8
:102D7000FF920F931F938C016BE9E62E64E0F62E11
:102D8000C701612F70E04AE050E00E946A1DC70150
:102D90006EE20E94A91C54E0169507955A95E1F73A
:102DA0000F701070C701B8014AE050E00E946A1D20
:102DB0001F910F91FF90EF900895A2E2B0E0E3EE33
:102DC000F6E10C94A9208E010F5F1F4F80E1D8011E
:102DD0001D928A95E9F78BE994E066E371E00E9421
:102DE000ED1D0E94DC0E20EC3DE948E555E32F8FF8
:102DF00038A349A35AA380EC97EFAAEBB7E38B8FD4
:102E00009C8FAD8FBE8F24EF31E040E050E02F8BE0
:102E1000388F498F5A8FA0E5CA2EA3ECDA2EE12C09
:102E2000F12CF0EC4F2EFDE95F2EF8E56F2EF5E367
:102E30007F2E88249924540133241E8A1D8A198ADE
:102E40001A8A1B8A1C8AFFC08BE994E00E946C1FBF
:102E50008434B9F0853430F48332B9F18C3209F01E
:102E6000CCC044C0833509F0C8C02F8D38A149A11A
:102E70005AA1C901DA012C013D0188249924540189
:102E8000E2C08BE994E064E40E94A91C8BE994E021
:102E900040EC5DE968E575E32AE030E00E948D1DB5
:102EA0008BE994E06CE20E94A91C8BE994E040EC71
:102EB00057EF6AEB77E32AE030E00E948D1D8BE943
:102EC00094E06CE20E94C71CBEC019821A821B8269
:102ED0001C821D821E821F82188619861A861B86F6
:102EE0001C861D861E861F86188A3AC0339434E0DD
:102EF000331609F0A8C069817A818B819C8128EE04
:102F000033E040E050E00E9439206F8F78A389A31E
:102F10009AA36D817E818F8198850E9439206B8F65
:102F20007C8F8D8F9E8F89859A85AB85BC858F8B95
:102F3000988FA98FBA8F6D857E858F8598890E941D
:102F400039206B017C0190E2C9169EE4D90690E01D
:102F5000E90690E0F90630F48CE162E30E94180380
:102F6000332471C0A0E3CA16A5E7DA06A0E0EA069A
:102F7000A0E0FA0618F48CE162E2F0CFB0E4CB16E0
:102F8000BCE9DB06B0E0EB06B0E0FB0618F48CE130
:102F900066E2E4CFE0E5CE16E3ECDE06E0E0EE0626
:102FA000E0E0FE0618F48CE162E1D8CFF0E6CF163F
:102FB000FAEEDF06F0E0EF06F0E0FF0618F48CE131
:102FC00065E1CCCF20E7C21621E1D20621E0E2067E
:102FD00020E0F20618F48CE161E0C0CF30EAC316BD
:102FE00036E8D30631E0E30630E0F30618F48CE16E
:102FF00063E0B4CF8CE165E0B1CFE0ED2E2E280E7A
:1030000049E0421500F1032D10E0000F111F000FE1
:10301000111F81E090E08C0F9D1F080F191FD80130
:103020006D917D918D919C912AE030E040E050E0DF
:103030000E943920620D711D811D911DF801608370
:103040007183828393838BE994E00E94321F892BE2
:1030500009F0FACE81149104A104B10489F4C301EA
:10306000B2010E94A90361E070E080E090E00E945C
:103070002B1BFFEFFE8B1D8A198A1A8A1B8A1C8A5A
:103080002F89388D498D5A8D82169306A406B50670
:10309000E0F40E94390329893A894B895C89280F19
:1030A000311D411D511D298B3A8B4B8B5C8B3D890A
:1030B000381708F48D8B4E89841708F48E8B08948A
:1030C000811C911CA11CB11C56C0C301B20128EE89
:1030D00033E040E050E00E946C208BE994E0BA01BC
:1030E000A9012AE030E00E945B1D8BE994E06CE2CC
:1030F0000E94A91C8BE994E06D894AE050E00E948F
:103100007B1D8BE994E06CE20E94A91C69897A8995
:103110008B899C89A50194010E946C208BE994E025
:10312000BA01A9012AE030E00E945B1D8BE994E01E
:103130006CE20E94A91C8BE994E06E894AE050E0A1
:103140000E947B1D8BE994E06CE20E94C71C4C0C32
:103150005D1C6E1C7F1C8B8D9C8DAD8DBE8D841572
:103160009505A605B70520F44F8C58A069A07AA054
:103170008824992454012F8D38A149A15AA1285E91
:1031800033404040504009F05ECFA296E2E10C94FB
:10319000C52080E065E970E042E050E00E94321A0C
:1031A0000895A1E0B0E0E7EDF8E10C94B92080E0EB
:1031B0000E94B1008DE061E00E94941B81E161E01A
:1031C0000E94941B0E94C70E80E060E00E94941B46
:1031D00081E061E00E94941B8BE994E040E052ECB6
:1031E00061E070E00E94AB1E0E9447110E94D00F68
:1031F0008BE994E063E471E00E94EA1D80E793E0CC
:103200000E94B7168BE994E06AE571E00E94EA1D1E
:103210008BE994E063E070E04AE050E00E94D61D44
:103220000E94C9187894439A86E067E00E947C1651
:10323000882329F043982D980E94DD16FBCF83E068
:1032400065E00E947C16882329F40E945611882389
:1032500009F000C18BE994E062E671E00E94EA1D8A
:1032600060E070E080E090E00E942A10882349F03E
:103270000E9451118BE994E06BE971E00E94ED1D11
:103280002D9A0E94DF0D22C08091E002833229F046
:103290008091E3028B7F8093E3028091E30281FFC0
:1032A00015C082FD13C064EF71E080E090E00E94E1
:1032B0002A10882359F00E9451118BE994E06BE9A0
:1032C00071E00E94ED1D0E94DF0D2D9A8091DF02BA
:1032D000823239F58091E002833219F581E00E9453
:1032E000980D8091E30282FF09C08BE994E066EBC0
:1032F00071E00E94ED1D0E941D0813C064E170E0A2
:1033000080E090E00E942B1B80E2BE016F5F7F4F48
:1033100041E021E00E949A08882319F481E080931B
:1033200084038BE994E061EC71E00E94EA1D8FE078
:103330000E94B10080E00E9413041092430380E0D9
:103340000E9423031092000490E0983158F4292F32
:103350002F5FE92FF0E0E051FD4F8785882311F0C2
:10336000922FF3CF9093000483E08093D4020E94C5
:10337000DC0E80918403882311F00E941F0A809143
:10338000E202883211F08A3239F48BE994E040E0AD
:1033900052EC61E070E02BC0893271F48BE994E06B
:1033A00040EA56E861E070E00E94AB1E8091C200E6
:1033B00080628093C20022C080911803887180319E
:1033C00069F04091F1025091F2026091F302709124
:1033D000F4024A3051056105710538F48BE994E037
:1033E00040E855E260E070E002C08BE994E00E94A2
:1033F000AB1E04C08BE994E00E946C1F8BE994E043
:103400000E94321F892BB1F78091E102843229F0AA
:103410008091C1008F7E8093C1008091E20285324D
:1034200029F08091C100877F8093C1001092FE0334
:103430001092FF03109282030E94051B60934403C5
:103440007093450380934603909347032196E2E0EF
:103450000C94D5200E94DF0D8091DF02823209F0AA
:1034600017CF12CF823000F5E82FF0E0EE0FFF1FEC
:10347000EA5FFB4F71836083882319F08130A1F4E8
:1034800008C0809169008C7F842B80936900E89A42
:10349000089580916900440F551F440F551F837F85
:1034A000842B80936900E99A08951F920F920FB6BA
:1034B0000F9211242F933F934F935F936F937F93BA
:1034C0008F939F93AF93BF93EF93FF9380910604E5
:1034D00090910704892B29F0E0910604F0910704EC
:1034E0000995FF91EF91BF91AF919F918F917F913E
:1034F0006F915F914F913F912F910F900FBE0F9061
:103500001F9018951F920F920FB60F9211242F93B0
:103510003F934F935F936F937F938F939F93AF935B
:10352000BF93EF93FF938091080490910904892B36
:1035300029F0E0910804F09109040995FF91EF91B9
:10354000BF91AF919F918F917F916F915F914F91BB
:103550003F912F910F900FBE0F901F9018951F92C3
:103560000F920FB60F9211242F933F938F939F9337
:10357000AF93BF9380910E0490910F04A09110041B
:10358000B0911104309112040196A11DB11D232F99
:103590002D5F2D3720F02D570196A11DB11D2093D1
:1035A000120480930E0490930F04A0931004B09320
:1035B000110480910A0490910B04A0910C04B09125
:1035C0000D040196A11DB11D80930A0490930B0474
:1035D000A0930C04B0930D04BF91AF919F918F9174
:1035E0003F912F910F900FBE0F901F9018958FB79E
:1035F000F89420910E0430910F04409110045091E2
:1036000011048FBFB901CA0108959FB7F8942091A2
:103610000A0430910B0440910C0450910D0486B5BE
:10362000A89B06C08F3F21F02F5F3F4F4F4F5F4F4A
:103630009FBF542F432F322F2227280F311D411DAA
:10364000511D82E0220F331F441F551F8A95D1F769
:10365000B901CA010895EF92FF920F931F93CF9380
:10366000DF937B018C010E94051BEB010EC00E94C1
:10367000051B6C1B7D0B685E7340C8F30894E10862
:10368000F10801091109C851DC4FE114F1040105E9
:10369000110569F7CDB7DEB7E6E00C94D1200197AC
:1036A00039F0880F991F880F991F02970197F1F73A
:1036B0000895789484B5826084BD84B5816084BDAA
:1036C00085B5826085BD85B5816085BDEEE6F0E09B
:1036D000808181608083E1E8F0E0108280818260F7
:1036E0008083808181608083E0E8F0E08081816078
:1036F0008083E1EBF0E0808184608083E0EBF0E0A8
:10370000808181608083EAE7F0E08081846080834B
:1037100080818260808380818160808380818068F5
:1037200080831092C1000895CF93DF93482F50E01B
:10373000CA0186569F4FFC0134914A575F4FFA01E8
:103740008491882369F190E0880F991FFC01E85962
:10375000FF4FA591B491FC01EE58FF4FC591D49154
:10376000662351F42FB7F8948C91932F9095892369
:103770008C93888189230BC0623061F42FB7F89451
:103780008C91932F909589238C938881832B8883A8
:103790002FBF06C09FB7F8948C91832B8C939FBF4B
:1037A000DF91CF910895833071F0843028F4813017
:1037B000A1F0823021F514C08630B1F08730D1F00D
:1037C0008430E9F404C0809180008F7703C0809139
:1037D00080008F7D80938000089584B58F7702C02C
:1037E00084B58F7D84BD08958091B0008F778093DC
:1037F000B00008958091B0008F7D8093B00008954F
:10380000FF920F931F93F62E482F50E0CA01825566
:103810009F4FFC012491CA0186569F4FFC011491D1
:103820004A575F4FFA0104910023C9F0222319F08F
:10383000822F0E94D31BE02FF0E0EE0FFF1FEE5807
:10384000FF4FA591B4919FB7F894FF2021F48C917C
:103850001095812302C08C91812B8C939FBF1F9167
:103860000F91FF9008950F931F93482F50E0CA01C6
:1038700082559F4FFC012491CA0186569F4FFC013F
:1038800004914A575F4FFA011491112319F420E073
:1038900030E015C0222319F0822F0E94D31B812F04
:1038A00090E0880F991F84589F4FFC01A591B49117
:1038B0008C9120E030E0802311F021E030E0C9015C
:1038C0001F910F910895982F8E3008F09E50977099
:1038D000809187028295880F880F807C892B809346
:1038E0007C0080917A00806480937A0080917A00D5
:1038F00086FDFCCF2091780040917900942F80E0E4
:1039000030E0282B392BC9010895A0E0B0E0EBE8A6
:10391000FCE10C94B3207C016B018A01C0E0D0E093
:103920000FC0D6016D916D01D701ED91FC91019011
:10393000F081E02DC7010995C80FD91F0150104033
:103940000115110571F7CE01CDB7DEB7E8E00C9493
:10395000CF20DC01ED91FC910190F081E02D0995E3
:103960000895EF92FF920F931F938C016DE00E94D8
:10397000A91C7C01C8016AE00E94A91C9C012E0DB3
:103980003F1DC9011F910F91FF90EF900895EF9295
:10399000FF920F931F937C010E94A91C8C01C70109
:1039A0000E94B11C9C01200F311FC9011F910F9172
:1039B000FF90EF900895CF93DF93EC0161157105AF
:1039C00019F420E030E00FC0DB010D900020E9F792
:1039D0001197A61BB70BE881F9810280F381E02DD6
:1039E000AD0109959C01C901DF91CF9108954F92D6
:1039F0005F927F928F929F92AF92BF92CF92DF920F
:103A0000EF92FF920F931F93DF93CF93CDB7DEB763
:103A1000A1970FB6F894DEBF0FBECDBF2C01742E58
:103A2000CB01223008F42AE019A231E2C32ED12CB6
:103A3000CC0EDD1E822E9924AA24BB24672D752F5F
:103A4000A50194010E946C2079018A01C801B70187
:103A5000A50194010E943920472D461B0894C108F6
:103A6000D1084A3010F4405D01C0495CF601408342
:103A7000E114F1040105110521F07E2C5F2DC80130
:103A8000DDCFC201B6010E94DB1CA1960FB6F894EF
:103A9000DEBF0FBECDBFCF91DF911F910F91FF9081
:103AA000EF90DF90CF90BF90AF909F908F907F90DE
:103AB0005F904F900895DC012115310541F4ED919F
:103AC000FC910190F081E02D642F099508950E94EA
:103AD000F71C0895EF92FF920F931F939A017B01B9
:103AE00000E010E0B801A7010E945B1D1F910F913B
:103AF000FF90EF900895EF92FF920F931F939A011A
:103B0000E62EFF2400E010E0B801A7010E945B1D33
:103B10001F910F91FF90EF900895A0E0B0E0E3E9CE
:103B2000FDE10C94B320EC016A017B012115310504
:103B300041F4E881F9810190F081E02D642F09952D
:103B40001BC02A303105B1F477FF13C06DE20E942B
:103B5000A91C8C0144275527BA014C195D096E092F
:103B60007F09CE012AE00E94F71C9C01200F311F23
:103B700004C02AE00E94F71C9C01C901CDB7DEB742
:103B8000E8E00C94CF20EF92FF920F931F937B01FC
:103B90009A010027F7FC0095102FB801A7010E9499
:103BA0008D1D1F910F91FF90EF900895EF92FF925E
:103BB0000F931F937C010E94C31D8C01C7010E94BB
:103BC000B11C9C01200F311FC9011F910F91FF9063
:103BD000EF9008950E94DB1C0895EF92FF920F93DF
:103BE0001F937C010E94EA1D8C01C7010E94B11C39
:103BF0009C01200F311FC9011F910F91FF90EF9081
:103C0000089508951F920F920FB60F9211242F93CB
:103C10003F934F938F939F93EF93FF938091C000B7
:103C200082FD1DC04091C600209153043091540480
:103C30002F5F3F4F2F733070809155049091560441
:103C40002817390771F0E0915304F0915404ED5EA8
:103C5000FB4F4083309354042093530402C080915F
:103C6000C600FF91EF919F918F914F913F912F91BE
:103C70000F900FBE0F901F9018951F920F920FB6C6
:103C80000F9211242F933F938F939F93EF93FF9362
:103C900020919704309198048091990490919A040E
:103CA0002817390731F48091C1008F7D8093C100BE
:103CB00014C0E0919904F0919A04E95AFB4F2081D5
:103CC0008091990490919A0401968F7390709093CB
:103CD0009A04809399042093C600FF91EF919F91DD
:103CE0008F913F912F910F900FBE0F901F901895BD
:103CF000A0E0B0E0EEE7FEE10C94AF20FC011382FF
:103D0000128288EE93E0A0E0B0E084839583A683DE
:103D1000B78388EC92E091838083758764875787A7
:103D20004687318B208B138B028BF58AE48AD78AE6
:103D3000C68AB18EA08E938E828E8F85848F88895D
:103D4000858F8989868F8A89878F8B8980A3209622
:103D5000ECE00C94CB20AF92BF92DF92EF92FF92F7
:103D60000F931F93CF93DF93EC017A018B01DD2436
:103D7000403081EE580780E0680780E0780711F056
:103D8000DD24D39491E0A92EB12CEC89FD89DD20AE
:103D900069F0C50108A002C0880F991F0A94E2F7D4
:103DA000808360E079E08DE390E005C0108260E8F8
:103DB00074E88EE190E0A80197010E946C202150E8
:103DC000304040405040569547953795279580E1C3
:103DD0002030380720F0DD2011F0DD24D6CFE8892F
:103DE000F9893083EA89FB89208319A2EE89FF894A
:103DF000408121E030E0C9010C8C02C0880F991F7E
:103E00000A94E2F7482B4083EE89FF894081C9017B
:103E10000D8C02C0880F991F0A94E2F7482B40834B
:103E2000EE89FF894081C9010E8C02C0880F991F5D
:103E30000A94E2F7482B4083EE89FF8980810F8C3A
:103E400002C0220F331F0A94E2F720952823208313
:103E5000DF91CF911F910F91FF90EF90DF90BF9076
:103E6000AF900895DC011C96ED91FC911D97E05CEC
:103E7000FF4F2191319180819181281B390B2F7344
:103E80003070C90108958BE994E00E94321F892B9C
:103E900011F00E94011E0895DC011C96ED91FC9129
:103EA0001D97E05CFF4F20813181E054F040DF013D
:103EB000AE5BBF4F8D919C9111972817390719F46C
:103EC0002FEF3FEF07C08D919C91E80FF91F808184
:103ED000282F30E0C9010895DC011C96ED91FC917A
:103EE0001D97E05CFF4F20813181E054F040DF01FD
:103EF000AE5BBF4F8D919C9111972817390719F42C
:103F00002FEF3FEF10C08D919C911197E80FF91F93
:103F100020818D919C91119701968F7390701196CD
:103F20009C938E9330E0C9010895DC0191968C91A9
:103F30009197882339F05496ED91FC9155978081A3
:103F400086FFF9CF91961C920895CF93DF93EC01F1
:103F5000EE85FF85E05CFF4F20813181E054F04029
:103F60002F5F3F4F2F733070DF01AE5BBF4F8D91DE
:103F70009C91119728173907D1F3E05CFF4F80819E
:103F80009181E054F040E80FF91F6083EE85FF85D2
:103F9000E05CFF4F31832083EE89FF89208181E03F
:103FA00090E00F8C02C0880F991F0A94E2F7282B2B
:103FB000208381E089A3EC89FD89808180648083EE
:103FC00081E090E0DF91CF9108958F929F92AF9220
:103FD000BF92CF92DF92EF92FF920F931F9300D088
:103FE00000D00F92EDB7FEB7319684E0ADB7BEB703
:103FF00011968C9383E0818387E0828385E08383BD
:1040000081E084838BE994E063E174E047E554E068
:1040100025EC30E004EC10E0B0ECEB2EF12CA1EC40
:10402000CA2ED12CF2ECAF2EB12CE6EC8E2E912CB8
:104030000E94781E0F900F900F900F900F901F917D
:104040000F91FF90EF90DF90CF90BF90AF909F9037
:104050008F900895CF93DF930E94591B0E94D1182F
:10406000C3E4DFE10E945F122097E1F30E94431F47
:10407000F9CF629FD001739FF001829FE00DF11D87
:10408000649FE00DF11D929FF00D839FF00D749FD2
:10409000F00D659FF00D9927729FB00DE11DF91F7E
:1040A000639FB00DE11DF91FBD01CF0111240895DB
:1040B000AA1BBB1B51E107C0AA1FBB1FA617B7074E
:1040C00010F0A61BB70B881F991F5A95A9F780956A
:1040D0009095BC01CD010895A1E21A2EAA1BBB1B2D
:1040E000FD010DC0AA1FBB1FEE1FFF1FA217B307C4
:1040F000E407F50720F0A21BB30BE40BF50B661FDA
:10410000771F881F991F1A9469F76095709580959D
:1041100090959B01AC01BD01CF01089597FB092E3D
:1041200005260ED057FD04D0D7DF0AD0001C38F486
:1041300050954095309521953F4F4F4F5F4F0895D3
:10414000F6F790958095709561957F4F8F4F9F4FB3
:1041500008952F923F924F925F926F927F928F922B
:104160009F92AF92BF92CF92DF92EF92FF920F9306
:104170001F93CF93DF93CDB7DEB7CA1BDB0B0FB610
:10418000F894DEBF0FBECDBF09942A8839884888CD
:104190005F846E847D848C849B84AA84B984C88463
:1041A000DF80EE80FD800C811B81AA81B981CE0F5A
:1041B000D11D0FB6F894DEBF0FBECDBFED0108953F
:1041C000EE0FFF1F0590F491E02D0994F894FFCFB6
:1041D00054582074696D656F757421005761697456
:1041E000696E672062696E640A00476F7420706BA5
:1041F000740A006461746120676F6F640A0052582A
:104200002068616E67007363616E6E6572206D6F0A
:104210006465004F70656E4C52536E672052582093
:104220007374617274696E672000206F6E20485746
:104230002000454550524F4D2064617461206E6FDF
:10424000742076616C6964206F722062696E6420EC
:104250006A756D70706572207365742C20666F725C
:1042600063696E672062696E640A005361766564F3
:104270002062696E64206461746120746F2045451A
:1042800050524F4D0A004920616D20736C61766574
:1042900000456E746572696E67206E6F726D616C39
:1042A000206D6F646500002100270520082B09227E
:1042B00009260A230A260B240C250C280C290C2A73
:1042C000C01200001A400AA1204EA5001B1E275252
:1042D0002C23308025000005400AA1204EA5002097
:1042E000244EA52C2330004B000006400AD0009D30
:1042F00049007B289D492C233000E1000005400A3D
:104300004501D7DC03B81E0EBF00232E48E801008C
:104310008A400A6001555502AD1E20000023C88066
:1043200025000005400AA1204EA50020244EA52C02
:10433000233000020002000200020002000200021C
:10434000000200020002000200020002000200025D
:1043500000028813409C08010305060708090A0BA0
:104360000C121300010000080000200000400000B3
:10437000800100000200000400000800001000009E
:1043800000100000200000000100000200070B0CDC
:104390001011150000000000A51F851C321F6C1FA6
:0443A0004C1F951FFA
:107E00000F92CDB7DEB7112484B714BE81FFF1D035
:107E100082E08093C00088E18093C10086E0809377
:107E2000C20080E18093C4008EE0CDD088249924E4
:107E3000CC24C394F5E0DF2EE1E1EE2E73E0F72EC3
:107E4000B6D0082F813479F4B2D08983C2D0898129
:107E5000823811F481E005C0813811F485E001C059
:107E600083E09ED09AC0823411F484E103C085344B
:107E700019F485E0B6D091C0853561F498D0082F0B
:107E800010E095D090E0982E8824802A912A880CC2
:107E9000991C82C0863521F484E0A3D080E0E1CF34
:107EA000843609F04CC083D082D0A82E80D0B82E62
:107EB00000E011E07CD0F80181938F01AE16D1F77C
:107EC00088D0FB2DF53489F4E0E0F1E00BC0F9999E
:107ED000FECF92BC81BC0894811C911C819180BD15
:107EE000FA9AF99AEA1598F358C08B2D863409F05E
:107EF00054C0F401F7BEE89507B600FCFDCFF401CD
:107F0000A0E0B1E02C9130E011968C91119790E0B7
:107F1000982F8827822B932B12960C01C7BEE895C9
:107F20001124329681E0A038B80761F7F401D7BE7A
:107F3000E89507B600FCFDCFE7BEE8952EC0843774
:107F4000F1F435D034D0182F32D0B82E42D0FB2DDA
:107F5000F63421F4F40105914F010CC0FB2DF534EA
:107F600049F4F999FECF92BC81BC0894811C911C04
:107F7000F89A00B5802F14D0115049F70EC08537FC
:107F800039F427D08EE10CD085E90AD08FE069CF93
:107F9000813511F488E017D01CD080E101D050CF9A
:107FA0009091C00095FFFCCF8093C600089580910A
:107FB000C00087FFFCCF8091C00084FD01C0A89560
:107FC0008091C6000895E0E6F0E098E19083808318
:107FD0000895EDDF803219F088E0F5DFFFCF84E10E
:107FE000DFCF1F93182FE3DF1150E9F7F2DF1F9166
:0E7FF0000895282E80E0E7DFEE27FF27099492
:027FFE0001057B
:0400000300007E007B
:00000001FF
